:040000007FEF04F09A
:10000800FACF13F0FBCF14F0E9CF15F0EACF16F0D2
:10001800E1CF17F0E2CF18F0D9CF19F0DACF1AF004
:10002800F3CF1BF0F4CF1CF0F6CF1DF0F7CF1EF086
:10003800F8CF1FF0F5CF20F0F294E30E026EE00E39
:10004800016EAEEC08F0000100018507D8A0860714
:100058000001000186518511D8A401D001D06DD0CE
:10006800000E00010001866F640E0001856F2BC031
:1000780027F02CC028F027500001000183272850C2
:10008800000100018423000100018451800A590FF6
:10009800100ED8B4835DD8A001D001D025D00001BE
:1000A800F00E00018327D80E00018423334A342A36
:1000B8003450800A7D0FE80ED8B4335CD8A001D044
:1000C80001D012D0180E3326FC0E34222250030A17
:1000D800E70ED8B42118D8B401D001D005D0214AF0
:1000E800222A02D001D000D024502310D8B401D045
:1000F80001D004D02306D8A0240600D038503710E9
:10010800D8B401D001D004D03706D8A0380600D022
:1001180036503510D8B401D001D004D03506D8A057
:10012800360600D026502510D8B401D001D005D00D
:100138002506D8A0260601D000D03D6601D001D002
:1001480087D0116E030E406E11502850800A7D0F23
:10015800E80ED8B4275CD8A001D001D064D0000E36
:10016800386E030E376E5FD05ED02850800A800F3D
:10017800640ED8B4275CD8B001D001D008D0000EE6
:1001880000010001826F0A0E0001816F61D027C053
:1001980008F028C009F0000E0B6E640E0A6E44ECDD
:1001A80007F008C081F009C082F052D051D0285021
:1001B800800A800F0A0ED8B4275CD8B001D001D0CD
:1001C80008D0000E00010001826F0A0E0001816F45
:1001D8003FD0000E046E640E036E27C001F028C0E5
:1001E80002F0F6EC07F001C008F002C009F0000EBA
:1001F8000B6E0A0E0A6E44EC07F008C081F009C0C5
:1002080082F026D025D027C001F028C002F0000EC9
:10021800046E0A0E036EF6EC07F001C081F002C00E
:1002280082F016D015D031C011F032C012F0125041
:10023800000AD8B401D00CD01150000AD8B495D710
:10024800010AD8B4B4D7030AD8B4DDD701D000D096
:100258003D50020AD8A401D001D06BD0116E000E17
:10026800406E11502850800A790FD00ED8B4275C00
:10027800D8A001D001D048D0000E386E030E376EDA
:1002880043D042D027C008F028C009F0030E0B6EF7
:10029800E80E0A6E44EC07F008C081F009C082F04D
:1002A80048D0030E046EE80E036E27C001F028C084
:1002B80002F0F6EC07F001C008F002C009F0000EE9
:1002C8000B6E640E0A6E44EC07F008C081F009C09A
:1002D80082F02FD0000E046E640E036E27C001F06A
:1002E80028C002F0F6EC07F001C008F002C009F0DF
:1002F800000E0B6E0A0E0A6E44EC07F008C081F07F
:1003080009C082F016D015D031C011F032C012F0F9
:100318001250000AD8B401D00CD01150000AD8B439
:10032800B1D7010AD8B4BDD7030AD8B4D3D701D0FE
:1003380000D03D04D8A401D001D0B2D02250800A08
:10034800800F640ED8B4215CD8A001D001D009D0A8
:10035800116E020E406E115021C029F022C02AF001
:100368008AD02250800A800F0A0ED8B4215CD8A007
:1003780001D001D023D0116E010E406E115021C062
:1003880001F022C002F0000E046E0A0E036E4AEC61
:1003980008F001C011F002C012F033C008F034C0F8
:1003A80009F0000E0B6E640E0A6E44EC07F008505C
:1003B8001124296E095012202A6E5DD0116E000E8C
:1003C800406E115021C001F022C002F0000E046EF0
:1003D800640E036E4AEC08F001C011F002C012F07E
:1003E80033C008F034C009F0000E0B6E0A0E0A6E16
:1003F80044EC07F008501124296E095012202A6E87
:100408003AD039D038D029C008F02AC009F0000EF7
:100418000B6E640E0A6E44EC07F008C081F009C048
:1004280082F03ED0000E046E640E036E29C001F007
:100438002AC002F0F6EC07F001C008F002C009F08B
:10044800000E0B6E0A0E0A6E44EC07F008C081F02D
:1004580009C082F025D029C001F02AC002F0000EA0
:10046800046E0A0E036EF6EC07F001C081F002C0BC
:1004780082F016D015D031C011F032C012F01250EF
:10048800000AD8B401D00CD01150000AD8B4BBD798
:10049800010AD8B4C7D7030AD8B4DDD701D000D031
:1004A80038503710D8B401D001D033D0116E030EB4
:1004B800406E115019D0000E00010001826F0A0E23
:1004C8000001816F26D0000E00010001826F000E2E
:1004D8000001816F1ED0000E00010001826F4C0EDA
:1004E8000001816F16D015D031C011F032C012F062
:1004F8001250000AD8B401D00CD01150000AD8B458
:10050800DAD7010AD8B4DFD7030AD8B4E4D701D0C0
:1005180000D036503510D8B401D001D0A4D0116E17
:10052800030E406E11503D6601D001D030D01AD074
:1005380019D0000E00010001826F0A0E0001816FC0
:1005480026D0000E00010001826F010E0001816FAC
:100558001ED0000E00010001826F410E0001816F64
:1005680016D015D031C011F032C012F01250000A66
:10057800D8B401D00CD01150000AD8B4DAD7010A87
:10058800D8B4DFD7030AD8B4E4D701D000D03D04EB
:10059800D8A401D001D030D01AD019D0000E000153
:1005A8000001826F0A0E0001816F26D0000E000143
:1005B8000001826F410E0001816F1ED0000E000104
:1005C8000001826F480E0001816F16D015D031C02E
:1005D80011F032C012F01250000AD8B401D00CD079
:1005E8001150000AD8B4DAD7010AD8B4DFD7030A01
:1005F800D8B4E4D701D000D03D50020AD8A401D025
:1006080001D031D01AD019D0000E00010001826F3C
:100618000A0E0001816F27D0000E00010001826FD1
:10062800020E0001816F1FD0000E00010001826FD1
:10063800410E0001816F17D016D031C011F032C0C1
:1006480012F01250000AD8B401D00DD01150000A8F
:10065800D8B4DAD7010AD8B4DFD7030AD8B4E4D7B4
:1006680002D001D000D026502510D8B401D001D036
:1006780034D01AD019D0000E00010001826F410E4B
:100688000001816F25D0000E00010001826F000E6D
:100698000001816F1DD0000E00010001826F050E60
:1006A8000001816F15D014D031C011F032C012F0A2
:1006B8001250000AD8B401D00BD01150000AD8B497
:1006C800DAD7010AD8B4DFD7030AD8B4E4D700D000
:1006D800116E020E406E115000D08A888B848B8276
:1006E80071D08A9C8A9E8B9E8B9C8B968B988B8ACA
:1006F800A0D08A8C8A9E8B9E8B8C8B868B888B8ACB
:1007080098D08A9C8A9E8B8E8B9C8B968B888B9A92
:1007180090D08A9C8A9E8B9E8B9C8B868B888B9A8A
:1007280088D08A8C8A9E8B9E8B8C8B868B988B9A92
:1007380080D08A9C8A8E8B9E8B9C8B868B988B9A7A
:1007480078D08A9C8A8E8B9E8B9C8B968B988B9A62
:1007580070D08A9C8A9E8B9E8B8C8B868B988B8A7A
:1007680068D08A9C8A9E8B9E8B9C8B968B988B9A42
:1007780060D08A9C8A9E8B9E8B9C8B868B988B9A4A
:1007880058D08A8C8A8E8B8E8B8C8B868B888B8AA2
:1007980050D08A9C8A9E8B9E8B8C8B968B988B9A3A
:1007A80048D08A8C8A9E8B9E8B8C8B968B988B9A42
:1007B80040D08A8C8A8E8B8E8B9C8B968B988B8A5A
:1007C80038D037D0000181C011F0000182C012F08A
:1007D8001250000AD8B401D02CD01150000AD8B455
:1007E80080D7010AD8B485D7030AD8B48AD7010AB2
:1007F800D8B48FD7070AD8B494D7010AD8B499D7F0
:10080800030AD8B49ED7010AD8B4A3D70F0AD8B41C
:10081800A8D7010AD8B4ADD7030AD8B4B2D74B0ABF
:10082800D8B4B7D7090AD8B4BCD7040AD8B4C1D742
:1008380000D040C011F0126A11BE120632501218D0
:1008480002E131501118D8A401D001D002D08A9AFF
:1008580010D08A8A0ED00DD08A888B848B921DD0B6
:100868008A988B848B8219D08A888B948B8215D036
:1008780014D031C011F032C012F01250000AD8B4AE
:1008880001D00BD01150000AD8B4E6D7010AD8B469
:10089800E7D7030AD8B4E8D700D0314A322A325011
:1008A800800A800F030ED8B4315CD8A001D001D0E3
:1008B80005D0000E326E000E316E00D020C0F5FF5C
:1008C8001FC0F8FF1EC0F7FF1DC0F6FF1CC0F4FFD5
:1008D8001BC0F3FF1AC0DAFF19C0D9FF18C0E2FF26
:1008E80017C0E1FF16C0EAFF15C0E9FF14C0FBFFFF
:1008F80013C0FAFF11007EEF08F0600ED36E180ED9
:100908007E6E000E7F6E110EC26E000EC16EAE0EB0
:10091800C06E180E926E000E936E010E946EF19ECC
:100928007786000E00010001866F640E0001856F56
:10093800000E326E000E316E000E00010001846F51
:10094800000E0001836F000E346E000E336E000E31
:10095800226E000E216E000E246E000E236E000E15
:10096800286E000E276E00017B6F030E406E00019B
:100978007B51000E366E000E356E000E386E000E7E
:10098800376E80B601D001D005D0000E266E060E57
:10099800256E05D0000E266E000E256E00D00001D3
:1009A8007B6F000E3D6E00017B5100017B6F9F0E37
:1009B80000010001606F00017B51000169EC08F043
:1009C800E30E00010001616FE00E0001606F00019D
:1009D8009CEC08F0F28AF28E00D0000E3A6E000EFF
:1009E800396E000E2E6E000E2D6E2E50800A800F6E
:1009F800100ED8B42D5CD8A001D001D002D02FD0D1
:100A08002ED000017B6F9F0E00010001606F000176
:100A18007B5100018EEC08F0BBEC08F001D000D04F
:100A2800B7EC08F00009D8A401D001D0F9D700D05C
:100A38000001A5EC08F00001000160513926000111
:100A4800000161513A222D4A2E2A2E50800A800F29
:100A5800100ED8B42D5CD8A001D001D0D2D739C09F
:100A68002FF03AC030F0000E3A6E000E396E000ECC
:100A78002E6E000E2D6E2E50800A800F100ED8B4E8
:100A88002D5CD8A001D001D002D02FD02ED00001EB
:100A98007B6FA70E00010001606F00017B51000110
:100AA8008EEC08F0BBEC08F001D000D0B7EC08F0F1
:100AB8000009D8A401D001D0F9D700D00001A5ECD5
:100AC80008F0000100016051392600010001615160
:100AD8003A222D4A2E2A2E50800A800F100ED8B4A2
:100AE8002D5CD8A001D001D0D2D739C03EF03AC091
:100AF8003FF0D00E00010001646F070E0001656F22
:100B0800000E0001666F000E0001676F00013EC015
:100B180060F000013FC061F00001000E000161BFFC
:100B2800FF0E0001626F0001636F0001A2EC07F085
:100B380060C06CF061C06DF062C06EF063C06FF0B1
:100B4800610E00010001706F3D0E0001716F000E13
:100B58000001726F000E0001736F000158EC06F07F
:100B68006CC03EF06DC03FF0F80E00010001646FEC
:100B78001F0E0001656F000E0001666F000E000178
:100B8800676F00013EC060F000013FC061F00001E6
:100B9800000E000161BFFF0E0001626F0001636F6C
:100BA8000001A2EC07F060C07BF061C07CF062C07D
:100BB8007DF063C07EF000012FC064F0000130C0FA
:100BC80065F00001000E000165BFFF0E0001666FB1
:100BD8000001676F00013EC060F000013FC061F096
:100BE8000001000E000161BFFF0E0001626F0001ED
:100BF800636F0001A2EC07F00001000160510001E1
:100C08007B25000100016C6F0001000161510001AA
:100C18007C2100016D6F00010001625100017D21FE
:100C280000016E6F00010001635100017E21000187
:100C38006F6FF00E00010001706F3F0E0001716FC1
:100C4800000E0001726F000E0001736F000158EC76
:100C580006F06CC02BF06DC02CF080B601D001D02E
:100C6800BCD624502310D8A401D001D0B6D6000E8B
:100C7800246E020E236E000E366E020E356E3D2A6D
:100C88003D50800A7D0FD8A001D001D0A6D6000122
:100C98007B6F000E3D6E00017B519FD69ED69DD680
:100CA8009CD69BD67FEF04F00001746F000E000104
:100CB8000001766F000174510001000173AF01D08B
:100CC80001D019D000010001731F0001721F00013B
:100CD800711F0001706D000E000171230001722365
:100CE800000173230001746F010E00010001766F8B
:100CF8000001745100D0000100016FAF01D001D094
:100D080015D0000100016F1F00016E1F00016D1F4B
:100D180000016C6D000E00016D2300016E230001BF
:100D28006F23010E00010001761B00D0000E0001A8
:100D38000001776F000E0001786F000E0001796FD7
:100D4800000E00017A6F00010001735170117111DA
:100D58007211D8B401D001D071D00001746F010EA6
:100D680000010001756F000174510ED00001D89088
:100D780000017037000171370001723700017337C5
:100D880000010001752B00D00001000173AF01D0F4
:100D980001D0ECD701D000D00001D89000017737FE
:100DA800000178370001793700017A370001000126
:100DB8007051000100016C5D0001000171510001DA
:100DC80000016D59000100017251000100016E59C6
:100DD800000100017351000100016F59D8A001D032
:100DE80001D01CD0000100017051000100016C5FAE
:100DF800000100017151000100016D5B000100015B
:100E08007251000100016E5B000100017351000185
:100E180000016F5B00010001778100D00001D890CC
:100E28000001733300017233000171330001703324
:100E380000010001752FB0D701D000D000010001DA
:100E48007651D8B401D001D011D0000100017A1F29
:100E58000001791F0001781F0001776D000E000165
:100E680078230001792300017A2300D077C06CF041
:100E780078C06DF079C06EF07AC06FF000D01200C3
:100E88000C6E000E0E6E0C500BAE01D001D009D0C6
:100E98000A6C0B1ED8B00B2A0C6E010E0E6E0C508D
:100EA80000D009AE01D001D007D0086C091ED8B017
:100EB800092A010E0E1A00D0000E106E000E0F6ED9
:100EC8000B500A10D8B401D001D028D00C6E010EF6
:100ED8000D6E0C5005D0D8900A360B360D2A00D06E
:100EE8000BAE01D001D0F7D701D000D0D8900F3683
:100EF80010360A50085C0B500958D8A001D001D010
:100F080006D00A50085E0B50095A0F8000D0D890BE
:100F18000B320A320D2EEAD701D000D00E50D8B4C9
:100F280001D001D005D00F6C101ED8B0102A00D007
:100F38000FC008F010C009F000D01200000E000128
:100F48000001686F000E0001696F000E00016A6FF2
:100F5800000E00016B6F00D00001000160A101D0FC
:100F680001D019D000010001645100010001682777
:100F78000001000165510001000169230001000121
:100F88006651000100016A23000100016751000158
:100F980000016B2300D00001D890000164370001E4
:100FA800653700016637000167370001D8900001F6
:100FB80063330001623300016133000160330001D3
:100FC80000016351601161116211D8A401D001D0F0
:100FD800C3D768C060F069C061F06AC062F06BC0D6
:100FE80063F01200056E000E076E055002AE01D0C8
:100FF80001D009D0016C021ED8B0022A056E010E7C
:10100800076E055000D004AE01D001D005D0036CA6
:10101800041ED8B0042A00D004500310D8B401D05C
:1010280001D024D0056E010E066E055005D0D8906B
:1010380003360436062A00D004AE01D001D0F7D713
:1010480001D000D00350015C04500258D8A001D050
:1010580001D005D00350015E0450025A00D0D89048
:1010680004320332062EEED701D000D00750D8B490
:1010780001D001D005D0016C021ED8B0022A00D0E0
:1010880001C001F002C002F000D01200000E066E8E
:10109800000E056E00D001A001D001D005D003508C
:1010A80005260450062200D0D89003360436D8907E
:1010B8000232013202500110D8A401D001D0EBD77E
:1010C80005C001F006C002F01200000100016051E5
:1010D8007F0BD56E000ED76E000ED66EF29400010F
:1010E800000160AF01D001D002D0F28A01D0F29A9B
:1010F800D58E12000001846B836B826B816B806BD1
:101108007F6B00EE21F01F0EEE6AE806FDE100019C
:1011180081EF04F0C2CF61F0C30E00016117000136
:101128000001D89060313C0B00016111C26E1200C1
:1011380060C062F061C063F063C0D7FF62C0D6FFD1
:101148001200C45000010001616FC3500001606FBC
:1011580000D0120001C003F002C004F004C0D7FFA1
:1011680003C0D6FF1200C230010B00D01200C282A9
:02117800120063
:020000040030CA
:0E00000000083900FF0080FF03C003E003404A
:00000001FF
